:100000000C94DB030C94F8030C94F8030C94F803A1
:100010000C94F8030C94F8030C94F8030C94F80374
:100020000C94F8030C94F8030C94FA210C94CC2251
:100030000C94611C0C94F8030C94F8030C94F803D2
:100040000C94F8030C94F8030C94F8030C94F80344
:100050000C94F8030C94E91C0C94F8030C94F8032A
:100060000C94F8030C94F8030C94F8030C94F80324
:100070000C94F8030C94F8030C94F8030C94F80314
:100080000C94F8030C94F8030C94F8030C94F80304
:100090000C94F8030C94F8030C94F8030C94F803F4
:1000A0000C94F8030C94F8030C94F803ED07ED0797
:1000B000190819088108AC09AC09AC099F0838096E
:1000C0004909490939236023582460235824AC2363
:1000D000CF2358242624352400574A004B004C00D7
:1000E0004D004E00000052000000500051004F0033
:1000F00001004800A90028004700AA0000000100F4
:10010000000001000100010001000100A900A80099
:100110000100AA0000002C000000BC00AE00BB00E3
:1001200044454255473A2064697361626C65642EA8
:100130000A0044454255473A20656E61626C656429
:100140002E0A000A0025303258006C65645F746125
:10015000736B3A20004F6E6573686F743A20616369
:10016000746976653A2025640A000A0025303862F1
:10017000003A200025303258000A722F63203031B7
:100180003233343536370A003F00433E20004C25D9
:10019000640A000A092D20537461747573202D0AB6
:1001A000686F73745F6B6579626F6172645F6C65B1
:1001B000647328293A20253032580A6B6579626FBA
:1001C0006172645F70726F746F636F6C3A20253078
:1001D00032580A6B6579626F6172645F69646C653D
:1001E0003A20253032580A74696D65725F72656114
:1001F00064333228293A202530386C580A000A091D
:100200002D2056657273696F6E202D0A5649443A47
:100210002030784645454428656D646172636865A1
:100220007229205049443A20307830303030284EFE
:10023000617669313029205645523A203078303085
:1002400030320A4255494C443A2020284665622003
:1002500032382032303232290A4F5054494F4E53EF
:100260003A204C5546412045585452414B4559205F
:10027000434F4E534F4C4520434F4D4D414E44202C
:10028000343039360A4743433A20352E342E302055
:100290004156522D4C4942433A20322E302E3020C6
:1002A0004156525F415243483A20617672350A0006
:1002B0000A092D20436F6E736F6C65202D0A45531C
:1002C000432F713A09717569740A000A092D204D8E
:1002D00061676963202D0A443A09446562756720A5
:1002E0004D65737361676520546F67676C650A5865
:1002F0003A094D6174726978204465627567204DD2
:100300006F646520546F67676C65202D2053686F9C
:1003100077206B65797072657373657320696E20E1
:100320006D617472697820677269640A4B3A094B8F
:100330006579626F61726420446562756720546FED
:1003400067676C65202D2053686F77206B65797027
:1003500072657373207265706F72740A4D3A094446
:1003600065627567204D6F75736520546F67676CA4
:10037000650A563A0956657273696F6E0A533A09EF
:100380005374617475730A433A0941637469766101
:10039000746520436F6E736F6C65204D6F64650AE2
:1003A00046312D4631303A095377697463682074B9
:1003B0006F204C6179657220302D3920284631300C
:1003C000203D204C30290A302D393A095377697481
:1003D000636820746F204C6179657220302D390A72
:1003E00047524156453A0953776974636820746FE0
:1003F000204C6179657220302028616C7465726EC2
:10040000617465290A423A094A756D7020746F203B
:10041000426F6F746C6F616465720A4553433A09A9
:100420004A756D7020746F20426F6F746C6F6164D9
:1004300065722028616C7465726E617465290A4565
:100440003A095072696E7420454550524F4D205301
:10045000657474696E67730A4253504143453A09A3
:10046000436C65617220454550524F4D0A006B65E3
:10047000796D61705F636F6E6669672E7261773A3E
:1004800020253032580A2E737761705F636F6E7467
:10049000726F6C5F636170736C6F636B3A2025756C
:1004A0000A2E636170736C6F636B5F746F5F636F51
:1004B0006E74726F6C3A2025750A2E737761705FC7
:1004C0006C63746C5F6C6775693A2025750A2E73CE
:1004D0007761705F7263746C5F726775693A20252B
:1004E000750A2E737761705F6C616C745F6C6775F1
:1004F000693A2025750A2E737761705F72616C749A
:100500005F726775693A2025750A2E6E6F5F677591
:10051000693A2025750A2E737761705F677261767C
:10052000655F6573633A2025750A2E737761705F86
:100530006261636B736C6173685F6261636B73703C
:100540006163653A2025750A2E6E6B726F3A20251D
:10055000750A0064656275675F636F6E6669672E12
:100560007261773A20253032580A2E656E61626CCE
:10057000653A2025750A2E6D61747269783A2025D6
:10058000750A2E6B6579626F6172643A2025750A6F
:100590002E6D6F7573653A2025750A006565636F6A
:1005A0006E6669673A0A64656661756C745F6C6152
:1005B0007965723A2025750A003F000A6D6F7573E0
:1005C000653A206F66660A000A6D6F7573653A209A
:1005D0006F6E0A000A6B6579626F6172643A206F10
:1005E00066660A000A6B6579626F6172643A206F11
:1005F0006E0A000A6D61747269783A206F66660A45
:10060000000A6D61747269783A206F6E0A000A649C
:10061000656275673A206F66660A000A64656275EE
:10062000673A206F6E0A000A0A4A756D70696E6734
:1006300020746F20626F6F746C6F616465722E2E10
:100640002E2000433E2000436C656172696E672076
:10065000454550524F4D0A000A00253032582000BF
:100660006B6579626F6172645F7265706F72743A04
:1006700020005B735D005B575D005B535D005B5268
:100680005D005B445D005B435D000E034E00610056
:1006900076006900310030000000140365006D0031
:1006A0006400610072006300680065007200000071
:1006B0000403090409025B00030100A0FA09040015
:1006C000000103010100092111010001224000077E
:1006D000058103080001090401000103000000096D
:1006E00021110100012232000705820320000109C7
:1006F000040200020300000009211101000122226E
:1007000000070583032000010705030320000112F1
:1007100001000200000008EDFE00000200010200DE
:10072000010631FF0974A1010975150026FF009526
:1007300020750881020976150026FF0095207508AE
:100740009102C005010980A101850319012AB700A2
:10075000150126B700950175108100C0050C09012F
:10076000A101850419012AA002150126A002950104
:1007700075108100C005010906A101050719E029CE
:10078000E71500250195087501810295017508811D
:10079000010507190029FF150026FF0095067508B9
:1007A000810005081901290595057501910295013A
:1007B00075039101C00011241FBECFEFDAE0DEBF48
:1007C000CDBF11E0A0E0B1E0ECEDF9E402C005908E
:1007D0000D92A43AB107D9F722E0A4EAB1E001C032
:1007E0001D92A035B207E1F70E94C6150C94EC24C7
:1007F0000C940000FF93EF93E091A401F091A50108
:10080000309709F00995EF91FF910895FC018591CA
:10081000803011F0EFDFFBCF0895FF27E0E230E2F8
:1008200047FF0CC0419597FF09C0EDE260957095B8
:1008300080959095611D711D811D911D27FF02C03E
:10084000219530E350E2AA27660F771F881F991F72
:10085000AA1FA41710F0A41B63955A95A9F7AA30F4
:1008600008F0A95FA05DAF93F3956115710581054F
:10087000910541F7ED3211F4EF93F395F21718F467
:100880003F93F395FBCF8F91B5DFFA95E1F708958C
:10089000E991F9918591803021F0853219F0AADF34
:1008A000F9CF089520E0E89455915532C1F35033C3
:1008B00011F4689455915A3348F4505390F3220F31
:1008C000022E220F220F200D250FF4CF0EF42195BA
:1008D00089919991533619F3533729F1533559F1C9
:1008E000BC0188279927E8945C3621F48991999175
:1008F00068945591543639F446EF7EF077FF0DC079
:100900008FEF9FEF0AC055374AE039F0583540E184
:1009100021F0523642E009F00895FF93EF937DDF16
:10092000EF91FF91B7CFFF93EF93FC01819180305E
:10093000B9F360DFFBCFFF93EF9368DFF1CFDF9375
:10094000CF93CDB7DEB72596A3DFCF91DF91089582
:10095000259A2D9A0C949714809117019091180163
:10096000029719F481E00E94310B10921801109245
:1009700017010895FC012081213031F482858823FC
:1009800031F082E090E0089588E090E0089581E001
:1009900090E008950E94BA04909318018093170183
:1009A0008130910519F0029781F0089582E00E944C
:1009B000F00A882329F082E00E94310B2D9A0895D5
:1009C00082E00E94100B2D98089581E00C94100B8A
:1009D00081E0089581E008950C94EA0408950C9450
:1009E000EE041F93CF93DF9300D000D01F92CDB7BA
:1009F000DEB749835A836B833091A70189819A813D
:100A0000311114C0662359F0222349F00E94050CCD
:100A1000182F682F89819A810E94AE0B03C00E9413
:100A2000D90B182F69817A81812F04C00E94050C8F
:100A300069817A810F900F900F900F900F90DF9146
:100A4000CF911F910C942713FC01262F40815181D7
:100A50006281738184810C94F10481E00895CF93C5
:100A6000DF93EC0160E00E942405BE01DF91CF918D
:100A70000C94EF040C94A8040C94951408950E940F
:100A8000380A0E943E052FEF84E39CE0215080400D
:100A90009040E1F700C000000C940F1D0F931F93CE
:100AA000CF93DF938C0161E00E942405EC01B80133
:100AB0000E94531AB801CE010E94EC04882309F465
:100AC00062C0B801CE010E949E1A882309F45BC05F
:100AD000B801CE010E949F19882309F454C0B801BF
:100AE000CE010E94D315882309F44DC0B801CE0170
:100AF0000E94FB18882309F446C0F80182818823EC
:100B0000D9F1CF3D8CE5D80779F140F4C115FCE56A
:100B1000DF0791F0C130DC4591F02EC0CC35EDE51A
:100B2000DE0741F1CD35FDE5DF0709F1CB35DD45C8
:100B300019F50E949F1020C00E943F0524C080919B
:100B40001202C82FC095C170C0FB80F980931202B9
:100B5000CC2329F082E391E00E94060414C080E2D5
:100B600091E00E94060410C00E944D110CC00E942A
:100B7000961002C00E94A210C801DF91CF911F9170
:100B80000F910C94E804C0E08C2FDF91CF911F915E
:100B90000F9108950E94441C0C94F5050E94F805DD
:100BA0000C944A1C8295982F937344E0949F900173
:100BB00011248C7C86958695282B822F8575880F2D
:100BC0002A7A2695822B089508950C94E40581E0F5
:100BD00008950C94E7050895CF93C82F0E94E5056A
:100BE0008C2F0E94E905CF91089580E00C94EC05CC
:100BF0000E94591B0C94EC05CF930E94591BC82FDF
:100C00008091A601C81741F1C093A60180911202FC
:100C100082FF1EC080FF04C08AE491E00E940604A7
:100C20008091120280FF0CC01F92CF9385E491E067
:100C30009F938F930E949F040F900F900F900F909F
:100C40008091120280FF04C083E491E00E940604B8
:100C50008C2FCF910C94EC05CF910895CF93DF9317
:100C6000CDB7DEB72B970FB6F894DEBF0FBECDBF62
:100C70004F83588769877A878B8761110E94CE0FCF
:100C80009E012F5F3F4F86E0F90111928A95E9F7A7
:100C900085E0FE013796D90101900D928A95E1F722
:100CA00089819A814C815D81452B31F09F3F31F4E0
:100CB00091E08F3F19F403C091E001C090E090FFF4
:100CC00009C049815A816B817C818D819E810E94FE
:100CD000EC0E05C0C9010E942D058111F2CF2B96A3
:100CE0000FB6F894DEBF0FBECDBFDF91CF91089550
:100CF000FC01808191810E94470C0895CF93882345
:100D000009F4A1C0C82F8238C1F40E94591B81FD8B
:100D10009AC069E380911B0190911C010E941C1CE8
:100D20000E94F00F2FEF81EE94E021508040904020
:100D3000E1F700C0000069E319C0833801F50E94A3
:100D4000591B80FD80C063E580911B0190911C01BF
:100D50000E941C1C0E94F00F2FEF81EE94E02150A6
:100D600080409040E1F700C0000063E580911B01E6
:100D700090911C010E941E1CCF910C94F00F84389E
:100D8000C1F40E94591B82FD5EC067E480911B0183
:100D900090911C010E941C1C0E94F00F2FEF81EE0D
:100DA00094E0215080409040E1F700C0000067E4EB
:100DB000DDCF8CEF8C0F813AF8F48C2F0E94B218A3
:100DC000811141C06C2F80911B0190911C010E94E8
:100DD000E61B882349F06C2F80911B0190911C0128
:100DE0000E941E1C0E94F00F6C2F80911B0190919D
:100DF0001C010E941C1CC0CF80E28C0F883048F47C
:100E0000C77081E001C0880FCA95EAF70E94AE0F53
:100E1000B3CFEBE5EC0FE33040F4F0E0E65AFE4FE1
:100E2000808190E0CF910C94AE1BC85AC73158F422
:100E3000EC2FF0E0EE0FFF1FE45DFE4F808191810B
:100E4000CF910C94C41BCF910895882309F45BC003
:100E5000682F823879F40E94591B81FF54C069E3DE
:100E600080911B0190911C010E941C1C0E94F00F9C
:100E700069E310C08338B1F40E94591B80FF43C05E
:100E800063E580911B0190911C010E941C1C0E9433
:100E9000F00F63E580911B0190911C010E941E1CC4
:100EA0000C94F00F843879F40E94591B82FF2BC0F8
:100EB00067E480911B0190911C010E941C1C0E9400
:100EC000F00F67E4E7CF8CEF860F813A18F380E2EA
:100ED000860F883048F4677081E001C0880F6A95FA
:100EE000EAF70E94B40FDCCF8BE5860F833020F445
:100EF00080E090E00C94AE1B685A673120F480E0EB
:100F000090E00C94C41B08951F93CF93DF93182F88
:100F1000EB010E947E06209741F08FE99FE0019748
:100F2000F1F700C000002197F6CF812FDF91CF911C
:100F30001F910C942507893319F060E070E002C01E
:100F400060E570E00C948407882321F00E94AE0FC6
:100F50000C94F00F0895882321F00E94B40F0C9494
:100F6000F00F0895CF92DF92EF92FF920F931F93AD
:100F7000CF93DF937C01D62FC72FFC01128105810F
:100F800002950F700E94A40F8823B9F01123A9F0D5
:100F90008C2F807F803421F080E28D0F883068F0C4
:100FA0008091360282FD09C082E00E9450100E94AA
:100FB000A40F91E0D82ED92601C0D12CCC2EC294FA
:100FC0008FE0C8228C2D90E08C30910508F0C4C1D0
:100FD000FC01EA5AFF4F0C9497248C2F807FCF702E
:100FE000882311F0C295C07F112399F0CC2309F416
:100FF0009FC180E28D0F883010F0D11104C08C2F7A
:101000000E94AE0F03C08C2F0E94C10F0E94F00FF0
:101010008FC18D2F0E942507CC2309F49DC180E24A
:101020008D0F883038F1DD2329F18C2F0E94C70FF6
:1010300024C08C2F807FCF70803211F0C295C07F8A
:10104000DD2319F0D130A1F13DC08091360282FF3D
:1010500017C0112349F0CC2329F08C2F0E94AE0F2A
:101060000E94F00F80E065C180E00E942507CC233C
:1010700009F472C18C2F0E94B40F0E94F00F6CC152
:10108000112371F0002341F0013031F40E94D10F9F
:101090008C2B0E94D90F60C10E94D10F8C2B1DC0D8
:1010A000002319F0013009F457C10E94E60F25C052
:1010B000112321F0063008F04FC10EC0053008F0B2
:1010C0004BC11BC0112361F0002331F0F701858172
:1010D00080FF2EC18F7085838C2F0E94A4073CC196
:1010E000002359F0D93309F034C1FFEF07EE13E0C4
:1010F000F15000401040E1F72AC18C2F0E94AB074D
:101100002BC18C2F86958695837019F0813061F004
:1011100023C1112321F08D2F9C2F937002C080E0FA
:1011200090E00E94AE1B20C1112321F08D2F9C2F37
:10113000937002C080E090E00E94C41B15C18C2F08
:10114000837009F047C011110BC12D2F22952695F0
:101150002770220F220F6D2F6F70862F90E0A0E076
:10116000B0E0022E04C0880F991FAA1FBB1F0A946B
:10117000D2F7D4FF10C04FE050E060E070E004C050
:10118000440F551F661F771F2A95D2F7409550953B
:101190006095709503C040E050E0BA01C695C695D1
:1011A000C3708A019B01082B192B2A2B3B2BC901E9
:1011B000B801C23049F058F4C13019F00E94A40AB5
:1011C000CFC00E94920ACCC00E94B60AC9C00E9439
:1011D000900AC6C0112319F08C2F817001C086952A
:1011E000882309F4BDC02D2F229526952770220F44
:1011F000220F6D2F6F70862F90E0A0E0B0E0022EDE
:1012000004C0880F991FAA1FBB1F0A94D2F7D4FFEE
:1012100010C04FE050E060E070E004C0440F551F84
:10122000661F771F2A95D2F7409550956095709567
:1012300003C040E050E0BA01C695C695C3708A016C
:101240009B01082B192B2A2B3B2BC901B801C2305B
:1012500049F058F4C13019F00E94890B81C00E94F6
:10126000770B7EC00E949B0B7BC00E94CA0A78C08D
:10127000CF70112339F08C2F0E94100B8D2F0E94FC
:10128000A4076EC08D2F0E94AB078C2F0E94310BDC
:1012900067C0D23F21F128F4D03F41F0D13FC1F0E7
:1012A00043C0D33F19F1D43F79F03EC0112341F040
:1012B000053008F051C08C2F8F710E94560B4CC026
:1012C000063008F049C0F7CF8091360282FF18C07F
:1012D000112339F08C2F8F710E94100B3DC0112308
:1012E000C9F38C2F8F710E94310B36C0112329F066
:1012F0008C2F8F710E94FB0A2FC00E94D60A2CC02F
:10130000112349F0CF718C2F0E94100B63E08C2FBA
:101310000E94351021C081E00E9450100230E0F0A0
:1013200082E00E94501018C0112331F0002391F286
:101330008D2F0E947E0610C0002399F2D93349F404
:101340001FEF27EE33E0115020403040E1F700C09E
:1013500000008D2F0E94250788EF8C0D843020F42B
:101360000E94591B0E94EC05DD20C9F00E94A00FCD
:1013700080FD15C0F70112820E949A0F0E94100B87
:10138000C7010E94F0090E949A0FDF91CF911F912F
:101390000F91FF90EF90DF90CF900C94310BDF9185
:1013A000CF911F910F91FF90EF90DF90CF90089514
:1013B0000F931F93CF93DF93EC01688179818A812A
:1013C0000E94520C8C010E94AD0B0E947E0AB80153
:1013D000CE010E94B207DF91CF911F910F91089526
:1013E000CF93DF93EC01988189812B813C81232B62
:1013F00031F08F3F31F481E09F3F19F403C081E069
:1014000001C080E080FD1DC0CE010E944E0581110B
:1014100010C00E94A40F8823A1F08A81882389F03C
:101420008091360282FD0DC082E0DF91CF910C9455
:101430005010CE010E94D809CE01DF91CF910C94BB
:101440002F05DF91CF91089580E090E00E94AE1BC0
:1014500080E090E00E94C41B0E94CE0F0C94F00F1D
:1014600080911B0190911C010E94201C0C94240A65
:101470000E94BB0F0C94300A92959F70963079F0C1
:1014800010F4925001C09A50923068F4803F69F095
:1014900018F4883E40F409C0843F29F406C0883E11
:1014A00020F0813F11F080E0089581E00895FC0173
:1014B000808191810E94470C0E943C0A0895CF933D
:1014C000DF9300D000D01F92CDB7DEB70F900F9002
:1014D0000F900F900F90DF91CF910895CF93DF93EE
:1014E00000D000D000D0CDB7DEB726960FB6F89466
:1014F000DEBF0FBECDBFDF91CF910895089508954F
:101500000C947F0A0C94800A0E94820A6093B601B0
:101510007093B7018093B8019093B9010C94240A99
:101520000C94840A0F931F930091B6011091B70198
:101530002091B8013091B901602B712B822B932B34
:101540001F910F910C94840A0F931F930091B60181
:101550001091B7012091B8013091B9016023712336
:10156000822393231F910F910C94840A0F931F934E
:101570000091B6011091B7012091B8013091B901E5
:1015800060277127822793271F910F910C94840A5B
:101590000C947F0A0E94C80A6093B2017093B30151
:1015A0008093B4019093B5010C94240A60E070E03C
:1015B000CB010C94CA0A611571058105910529F4C6
:1015C00081E0442361F080E00895DC01CB0104C098
:1015D000B695A795979587954A95D2F78170089506
:1015E000482F6091B2017091B3018091B401909144
:1015F000B5010C94DB0A0F931F9341E050E060E0CB
:1016000070E08A019B0104C0000F111F221F331FCD
:101610008A95D2F7C901B8011F910F910C94CA0A9B
:101620000F931F9341E050E060E070E004C0440F6E
:10163000551F661F771F8A95D2F78091B20190914E
:10164000B301A091B401B091B5018A019B01082BAF
:10165000192B2A2B3B2BC901B8011F910F910C9418
:10166000CA0A0F931F9341E050E060E070E004C0AD
:10167000440F551F661F771F8A95D2F740955095E6
:10168000609570958091B2019091B301A091B401E1
:10169000B091B5018A019B01082319232A233B231A
:1016A000C901B8011F910F910C94CA0A0F931F939F
:1016B00041E050E060E070E004C0440F551F661F39
:1016C000771F8A95D2F78091B2019091B301A091D2
:1016D000B401B091B5018A019B01082719272A2777
:1016E0003B27C901B8011F910F910C94CA0A0F93AF
:1016F0001F930091B2011091B3012091B401309178
:10170000B501602B712B822B932B1F910F910C94A1
:10171000CA0A0F931F930091B2011091B301209157
:10172000B4013091B50160237123822393231F916B
:101730000F910C94CA0A0F931F930091B20110915C
:10174000B3012091B4013091B50160277127822740
:1017500093271F910F910C94CA0A0895292F220FE5
:10176000920F890FE82FE695E695E695877051E090
:1017700001C0550F8A95EAF785E0E89FF001112432
:10178000E855FE4F20E030E070E04081CB01022EB2
:1017900002C0969587950A94E2F781708195842717
:1017A0008523842781932F5F3F4F2530310569F7CB
:1017B0000895292F220F920F890F682F669566953D
:1017C0006695982F977085E0689FB001112440E0DE
:1017D00050E080E0FB01E40FF51FE855FE4F20814B
:1017E00030E0092E02C0369527950A94E2F7217061
:1017F0003327042E01C0220F0A94EAF7822B4F5F91
:101800005F4F4530510531F70895BF92CF92DF9277
:10181000EF92FF920F931F93CF93DF938C01C090B1
:10182000B201D090B301E090B401F090B501809185
:10183000B6019091B701A091B801B091B901C82A41
:10184000D92AEA2AFB2ACFE1D0E0D701C6010C2E23
:1018500004C0B695A795979587950A94D2F780FD11
:1018600004C0219790F7B12C07C0BC2EB8018C2F73
:101870000E943D130197A9F38B2DDF91CF911F910A
:101880000F91FF90EF90DF90CF90BF900895CF938E
:10189000DF93EC010E94050CBE010E943D13DF9115
:1018A000CF9108951F93CF93DF93EB019091A70100
:1018B000992321F0CB010E94470C13C0882349F0E3
:1018C000CB010E94050C182F682FCE010E94AE0B91
:1018D00004C0CB010E94D90B182FBE01812F0E949A
:1018E0003D13DF91CF911F9108951F93CF93DF9305
:1018F000C091BA0116E08091BB01C81799F0D0E001
:101900001C9FF0011D9FF00D1124E454FE4F4081F7
:10191000518162817381848195810E946E0A219632
:10192000C770E9CFDF91CF911F9108954091EC01ED
:101930005091ED016091EE017091EF018091F00105
:101940009091F1010C946E0AEF92FF920F931F9306
:10195000CF93DF938091F10182958F7009F065C07C
:101960008091EE01882309F460C08091BA01F09063
:10197000BB011091EC010091ED016091EF017091BC
:10198000F00191E01F3F09F090E0C0911901D09162
:101990001A01292F96E0E92E8F1509F446C061152A
:1019A000710521F00F3F21F030E003C031E001C0AC
:1019B000322F90E030FD36C0E89EF001E99EF00D38
:1019C0001124DF01A454BE4F11963C91119730139E
:1019D00029C03C91311326C012963C9112973111C7
:1019E00021C013964D915C911497461B570B4C17D1
:1019F0005D07C0F48091F1018F7080618093F101E7
:101A0000EF53FE4F80818F70806180838CEE91E078
:101A10000E94F009DF91CF911F910F91FF90EF90FD
:101A20000C94750C01968770B7CFDF91CF911F9101
:101A30000F91FF90EF9008959F92AF92BF92CF9237
:101A4000DF92EF92FF920F931F93CF93DF93CDB767
:101A5000DEB761970FB6F894DEBF0FBECDBF8C0125
:101A600085E0F801DE011D9601900D928A95E1F75F
:101A7000D8011296EC909091EC01E091ED0120914B
:101A8000EF013091F0012115310531F0EF3F31F4D4
:101A900081E09F3F19F403C081E001C080E0B82FCE
:101AA000B1709B2E80FD47C1D8014C9111965C917D
:101AB00011971396AD90BC9014978CEEC82E81E0D0
:101AC000D82EF090EE01B501621B730B2091190125
:101AD00030911A01FF2009F4D9C08091F1016217F9
:101AE000730708F095C0282F207F09F052C05E13BD
:101AF00013C0491311C0FE2CE1100EC08F7080611D
:101B00008093F1010E94960CC6010E94F009809119
:101B1000F101F80185834DC1AB2831F05F3F31F40D
:101B200081E04F3F19F403C081E001C080E080FDF7
:101B300003C081E08E2502C080E090E0F82FF170B4
:101B4000FF2E80FF1CC08091BA012091BB0136E0BE
:101B5000821709F40BC190E0389FF001399FF00D16
:101B60001124E454FE4F6181561306C06081461370
:101B700003C06281E61203C001968770E9CFFE2C94
:101B8000EE2009F416C18091F10181608093F1018A
:101B900054C05E1306C0491304C0E11002C0F8012E
:101BA00099C0C8010E94570A882361F1EE2051F1C3
:101BB0002091F101822F82958F7090E0029774F04E
:101BC0008091EC019091ED0198878F831986BB86F7
:101BD000AA862C87CE0107960E94F00986E0F801BC
:101BE000ACEEB1E001900D928A95E1F70E94A40C51
:101BF0000E94960C0AC05E1711F1C8010E94570A94
:101C000081112CC0C8010E94F009FF24F394D1C0B7
:101C1000282F207F81F77A2DB98AA88A6E2D89898D
:101C20000E945F0A8CEE91E00E94F00986E0D601E6
:101C30001D928A95E9F70E94960CF12CBAC04913BF
:101C4000DCCFE110DACFF8018583C8010E94F009EA
:101C500086E0D6011D928A95E9F7ABC0EE2091F29D
:101C60002091F101822F82958F7090E002970CF401
:101C7000B5CF8091EC019091ED019A8389831B820D
:101C8000BD82AC822E83CE010196A6CF6217730768
:101C900008F044C0FE2CEE2009F4B4CF5E1330C02F
:101CA00049132EC02091F10120FD21C0822F829581
:101CB0008F70482F50E041155105C9F0F801258378
:101CC0004F30510541F08F5F982F9295907F822F72
:101CD0008F70892B8583C8010E94F00986E0F80186
:101CE000ACEEB1E001900D928A95E1F73CC086E040
:101CF000F801ACEEB1E001900D928A95E1F759C080
:101D0000C8010E94570A811169CF8091F101816059
:101D10008093F101C8010E94F0094BC07A2DB98A65
:101D2000A88A6E2D89890E945F0A86E0D6011D92DD
:101D30008A95E9F718C0EE2009F464CFC8010E9423
:101D4000570AF82E882309F45DCF86E0F801ACEE3F
:101D5000B1E001900D928A95E1F78CEE91E00E943E
:101D600078060E94A40C0E94960C23C04D875E87C3
:101D70008D859E850E94470C292F22952F70223039
:101D800028F49F7039F0811105C00BC0243028F46D
:101D90009F7049F4805E883020F0C8010E94F009ED
:101DA0009F2CF92C06C0D80115969C91907F91F735
:101DB000F8CF8F2D61960FB6F894DEBF0FBECDBF62
:101DC000DF91CF911F910F91FF90EF90DF90CF9017
:101DD000BF90AF909F9008951F93CF93DF93CDB79F
:101DE000DEB72C970FB6F894DEBF0FBECDBF4F8382
:101DF000588769877A878B879C87CE0107960E94D0
:101E00001C0D8823D1F09F8188852A853B85232B53
:101E100031F08F3F31F481E09F3F19F403C081E03E
:101E200001C080E080FD47C04F81588569857A8573
:101E30008B859C850E946E0A3EC086E0FE01379627
:101E4000DE01119601900D928A95E1F7FF81E885F8
:101E50006A857B856115710531F0EF3F31F481E0D2
:101E6000FF3F19F403C081E001C080E080FD23C082
:101E70002091BB0130E0C9010196877099274091FC
:101E8000BA0150E084179507F1F1F983EA837D8365
:101E90006C8396E0929FD001939FB00D1124A454BF
:101EA000BE4FFE01319601900D929A95E1F7809315
:101EB000BB010E94750C16E08091BA019091BB01A4
:101EC000891771F1189FC001112484549E4F0E94FC
:101ED0001C0D882329F1E091BA011E9FF001112405
:101EE000E454FE4F408151816281738184819581E8
:101EF0000E946E0A8091BA0190E00196877099273E
:101F00008093BA01D9CF0E94380A1092BB01109277
:101F1000BA01ECEEF1E086E0DF011D928A95E9F767
:101F20002C960FB6F894DEBF0FBECDBFDF91CF91D8
:101F30001F9108958091FA0185958595859508955D
:101F40008091FA01877008959091FA01977081E06D
:101F500009F480E0089580910502089590910502AA
:101F6000892B80930502089580959091050289231D
:101F7000809305020895109205020895809104024D
:101F8000089590910402892B80930402089580950E
:101F90009091040289238093040208951092040210
:101FA00008958091FB01089508950C94D40F0C942A
:101FB000D50F9091360292FD08C09091FB019817C1
:101FC00021F08093FB010C94D70F08958091FB01C1
:101FD000882329F01092FB0180E00C94D70F08951C
:101FE000CF93DF93E0911B01F0911C0180910502DA
:101FF0008083E0911B01F0911C019081809104028B
:10200000892B80838091FB01882381F0E0911B0163
:10201000F0911C019081892B808380911B0190910C
:102020001C010E94DA1B81110E94E60FC0911B0166
:10203000D0911C0148E050E062EF71E0CE010E94B7
:102040009D24892B69F088E0FE01A2EFB1E00190A8
:102050000D928A95E1F7CE01DF91CF910C94651B2B
:10206000DF91CF9108950C94D40F9091360292FD98
:1020700010C098E0899F90011124262B2093FA012B
:102080000E94100B8091FA018595859585950C9499
:1020900033100C94100B1092FA0180E00C94331062
:1020A0002091FA01809582238093FA01982F9770EE
:1020B00099F430E0482F082E000C550B24173507F3
:1020C00059F09091360292FD07C0859585958595CA
:1020D0000E94310B0C944B100895CF9390913602CF
:1020E00092FB222720F92817F9F0C82F892FC0FB6F
:1020F00082F98093360280913502909136020E94D7
:10210000C91082E00E9450108091120280FF0CC022
:102110001F92CF9385E591E09F938F930E949F0438
:102120000F900F900F900F90CF91089580913602ED
:1021300082FB882780F991E089270C946D1081E05B
:102140000C946D1080E00C946D1080E090E00E9483
:10215000B22421E0893E9E4F09F020E0822F0895AD
:1021600082E090E00C94AA2483E090E00C94AA24EE
:10217000CF9384E090E00E94AA24C82F82E290E0EE
:102180000E94AA242C2F30E0A901582BCA01CF911C
:102190000895CF93C92F682F84E090E00E94B8245F
:1021A0006C2F82E290E0CF910C94B824AB01BC017B
:1021B0008FE090E00C94CA24AB01BC0183E190E075
:1021C0000C94CA2460E070E0CB010C94DC1060E059
:1021D00070E0CB010E94D6100C94E21069EE7EEF05
:1021E00080E090E00E94D62460E082E090E00E94CF
:1021F000B82460E083E090E00E94B8241092B60119
:102200001092B7011092B8011092B90160E084E019
:1022100090E00E94B82460E082E290E00E94B8243E
:1022200060E085E090E00E94B82460E086E090E005
:102230000E94B8246FEF87E090E00E94B82440E04D
:1022400050E0BA0188E090E00E94CA2460E08DE08E
:1022500090E00E94B82440E050E0BA0188E190E0AC
:102260000E94CA2460E087E190E00E94B82440E028
:1022700050E0BA018CE190E00E94CA2460E070E076
:1022800080E290E00E94D62440E050E0BA0188E16C
:1022900090E00E94CA240C94E7100C94EE10682F72
:1022A0008EE090E00C94B8240E94CE1C60930E0245
:1022B00070930F02809310029093110260930A02B0
:1022C00070930B0280930C0290930D02089585B7D2
:1022D000806885BF85B7806885BF089581E00895CF
:1022E0000C946E1108950C9472110C9472110C944C
:1022F00075110C9472110C9479110C9472110E9446
:10230000671185ED9EE10E944F1B0E947D110C9488
:102310007B110E9473110C9472110E941A140C9478
:10232000EB050E94B91C0E942C150E948D110C9483
:1023300077118F929F92AF92BF92CF92DF92EF92DE
:10234000FF920F931F93CF93DF93CDB7DEB72A97FA
:102350000FB6F894DEBF0FBECDBF0E944115982E78
:1023600081110E94541186E0A82E82E0B82E00E070
:1023700010E0802E802F0E943E14D82EF501C190CF
:102380005F01C826B1F40F5F1F4F0430110589F7B4
:102390008FEF89838A831B820E94C21C8160782F01
:1023A0009D838C8349815A816B818D810E942E0689
:1023B0002FC08091120281FD0E944414E12CFF2461
:1023C000F3948C2D8F21F1F00E947011882399F0E5
:1023D000EE828F82DF2081E009F480E088870E940E
:1023E000C21C8160782F9A8789874E815F816885BA
:1023F0008A850E942E06F801EA5FFD4F8081F8264B
:10240000F08206C0E394FF0CF3E0EF12DACFBBCF0B
:1024100081E0911001C080E02A960FB6F894DEBFEB
:102420000FBECDBFDF91CF911F910F91FF90EF9025
:10243000DF90CF90BF90AF909F908F9008950E94B3
:1024400099110E94FB1A0C94FC05CF93DF930E9414
:102450004213EC01811522E59207E8F5811531E57B
:10246000930708F0B6C0883E910528F5803E910597
:1024700008F0E9C0883A910570F4853A910508F0B2
:102480007AC08130910509F473C008F4D9C004976B
:1024900008F0D9C0D5C08F3B910508F0D1C0C85A0B
:1024A000D0E0CC0FDD1FC35ADE4F0990D881C02D7C
:1024B000CE019464C9C0811540E5940708F069C055
:1024C000811550E4950708F060C09A9581159F41E9
:1024D00008F4B9C0B5C0811536E5930728F5811514
:1024E00045E5940708F092C0811554E5950708F07A
:1024F00087C0AC0143705527282F26952695C11516
:10250000D34508F06CC081E090E002C0880F991FAD
:102510004A95E2F740E2249F90011124EC01C22B7E
:10252000D32BCE019C6890C081152AE5920780F4D8
:10253000811539E5930708F072C0811548E59407C5
:1025400008F47EC0D82FCC27CE01806F906A7CC063
:1025500090568115904208F073C08D2F8F710E94A4
:10256000D613DD27D0628F71AE01582BCA016CC023
:1025700081E090E069C0C55AD0E0C557DE4F888140
:10258000C82FD0E0CE0190645FC0DF70CE01906AAA
:102590005BC074E0969587957A95E1F7282F2370B4
:1025A0003C2F337081E090E002C0880F991F3A956C
:1025B000E2F79C68AC01522B9A019C2F9F70969574
:1025C000969550E2959FE0011124C9018C2B9D2B1B
:1025D0003BC0D82FCC27CE01816F906A35C081E0F7
:1025E00090E002C0880F991F4A95E2F750E2259FBC
:1025F00090011124EC01C22BD32BCE019A6824C088
:10260000D82FCC27CE01846F906A1EC00E94D613AB
:102610008F7190E0D82FCC27CE01906215C08F70BB
:102620000E94D61394E0D695C7959A95E1F7CF709E
:10263000D0E0DC2FCC27D0699E01282BC90104C033
:1026400080E090E001C0CE01DF91CF910895272F67
:1026500030E0F901EE0FFF1F2E0F3F1FF9019CE044
:10266000899FE00DF11D1124E60FF11DEE0FFF1FF4
:10267000E852FF4F8591949108950E9427130E947C
:10268000251208958238910569F1B0F481339105DE
:1026900009F46DC048F48932910509F463C08A32A7
:1026A000910509F469C008958533910509F455C071
:1026B00089339105B9F00895833E910569F138F4A5
:1026C000803E9105B1F0823E910509F10895863E64
:1026D0009105A9F1873E9105B9F1843E910509F074
:1026E00064C023C02091350220FD4FC021FD4DC0A4
:1026F00008958091350280FD44C08091360280FFAC
:1027000044C08091350284FD42C083EE4DC080916B
:10271000350282FF38C0F5CF8091350282FD33C08B
:102720008091360280FD31C0ECCF8091360281FF6E
:1027300032C08091350284FD2AC087EE35C0809179
:10274000350283FF26C0F5CF8091350283FD21C07D
:102750008091360281FD1FC0ECCF8091350285FD4E
:102760001CC01DC08091350285FD19C016C0809126
:10277000350286FD16C017C08091350286FD13C054
:1027800010C089E311C082EE0FC080EE0DC080E062
:102790000BC086EE09C084EE07C089E205C085E360
:1027A00003C08AE201C081E390E008959091350270
:1027B00092FF0DC0282F2871283019F4877F84607C
:1027C00006C0282F2471243011F48B7F886093FF7A
:1027D0000DC0282F2871283119F4877E846106C026
:1027E000282F2471243111F48B7E886120913602C8
:1027F00020FF0DC0382F3871383019F4877F816081
:1028000006C0382F3171313011F48E7F886021FF7E
:102810000DC0282F2871283119F4877E816106C0E8
:10282000282F2171213111F48E7E886194FD877EDD
:10283000089508950E94A510811102C00E944D11B3
:102840000E94B010809312020E94B810909336023A
:10285000809335020E9419140E94B410682F70E012
:1028600080E090E00E94900A6091B2017091B30103
:102870008091B4019091B5010C94C80AE82FF0E062
:10288000E55CFD4F80810895CF92DF92EF92FF9239
:102890000F931F93CF93DF9389E791E00E94060483
:1028A0008BE3E82E82E0F82EC0E0D0E094E7C92E5A
:1028B00091E0D92E0CE611E0DF93CF93DF92CF9217
:1028C0000E949F0481E791E00E940604F701819134
:1028D0007F010E94D2051F928F931F930F930E9436
:1028E0009F048AE691E00E94060421968DB79EB768
:1028F00008960FB6F8949EBF0FBE8DBFC430D105A9
:10290000D9F6DF91CF911F910F91FF90EF90DF905B
:10291000CF90089580EA8A95F1F7089500C0089550
:102920000C948A1408950C9492140C9493140C949F
:102930009214F894E82FE295EF70F0E031A1282F7F
:102940002F7081E090E001C0880F2A95EAF7982F58
:102950009095932391A392A1892B82A378940895B3
:10296000CF93DF93C1E9D1E089918F3F11F00E94AD
:10297000991481E0C539D807B9F784E90E94991400
:1029800086E60E94991481E3DF91CF910C9499140B
:10299000CF92DF92EF92FF920F931F93CF93DF932B
:1029A0008C01C62FD0E0CE018F569E4F7C01FC01DA
:1029B00090819F3F09F447C0D62EF894E92FE29505
:1029C000EF70F0E081A19F7021E030E001C0220FA4
:1029D0009A95EAF7822B81A382A12095282322A32E
:1029E00078940E948E14EEE8F1E041E951E031E084
:1029F000C12C21912F3F89F0A22FA295AF70B0E09A
:102A000090968C9190E02F7002C0959587952A95AD
:102A1000E2F780FD02C0832F01C080E0C82A330F97
:102A20004E175F0731F7F70180818F3F11F00E9449
:102A3000991461E0C11001C060E08D2D0E949014D6
:102A4000C00FD11FC882DF91CF911F910F91FF90CE
:102A5000EF90DF90CF9008950E94B01484E0EBE3F4
:102A6000F2E0DF01982F1D929A95E9F7E7E3F2E093
:102A7000DF011D928A95E9F784E00E9483150C948A
:102A80003A051F93CF93DF9300D000D0CDB7DEB7C8
:102A900019821A821B821C8210E0612FCE010196DE
:102AA0000E94C8141F5F1430C1F744E050E0BE011B
:102AB0006F5F7F4F87E392E00E949D2411E00097B3
:102AC00009F410E0892B61F089819A81AB81BC8186
:102AD0008093370290933802A0933902B0933A0260
:102AE000212F44E06BE372E087E392E00E948415BB
:102AF0000E943C05812F0F900F900F900F90DF9157
:102B0000CF911F9108950895FF920F931F93CF9334
:102B1000DF938C01F62ED72FC42F222349F081E0BA
:102B2000809315020E94C21C90931402809313029A
:102B3000809115028823C1F08091130290911402B4
:102B40000E94DA1C059780F0EF2DFD2FD8014C2F45
:102B500050E0CD01801B910B841795071CF48D91DB
:102B60008193F7CF10921502DF91CF911F910F91B2
:102B7000FF9008950E94511F0E9491110C945D1FB7
:102B80000E94611F0E941F120C947F1F0E94601CF4
:102B90000E94381F0E947F110E94BA150E94C01522
:102BA0000E948911FBCFCF93DF93EC01FB0182815F
:102BB000882309F43CC1C430FDE5DF0760F4CB3F56
:102BC0009CE5D90788F49E0122503C45243131050B
:102BD00008F02EC109C0C236EDE5DE0729F0C63A7D
:102BE000FDE5DF0709F024C10E94B810909336027A
:102BF00080933502C1318CE5D80709F4C6C008F0CE
:102C000042C0C930ECE5DE0709F49BC000F5C530D1
:102C10008CE5D80709F485C078F4C330ECE5DE070D
:102C200009F478C008F07AC0C230DC4509F0F5C07C
:102C3000809135028160EFC0C7309CE5D90709F467
:102C400078C008F07AC0809135028061E4C0CD3050
:102C5000FCE5DF0709F487C058F4CB309CE5D907C1
:102C600009F479C008F07BC08091350288606FC09C
:102C7000CF30FCE5DF0709F480C008F082C0809106
:102C80003502877FC8C0CE3F9CE5D90709F471C0E3
:102C900000F5C531FCE5DF0709F485C068F4C331F0
:102CA0009CE5D90709F475C008F095C00E94380A60
:102CB000809135028F77AFC0CC3FFCE5DF07A9F1EB
:102CC00008F054C0CB3FDC4509F0A7C08091360224
:102CD00040C0C230EDE5DE0709F489C058F4C115E3
:102CE0008DE5D80709F45AC008F069C08091360212
:102CF00082602FC0C236EDE5DE0709F47CC0C63A1B
:102D0000FDE5DF0709F481C0C330DD4509F085C06A
:102D100080E06EC08091350282607DC08091350276
:102D200016C080913502886076C08091360282603C
:102D30004FC08091350280626EC080913502806400
:102D40006AC00E94380A80913502806864C084603D
:102D500062C081603DC0809135028E7F5CC08091F1
:102D600035028D7F58C08091350216C080913602A1
:102D700018C0809136028D7F2BC0809135028F7EE6
:102D80004AC0809135028F7D46C0809135028F7B8D
:102D900042C080913502877F8B7F3DC08091360293
:102DA0008D7F8E7F15C08091350282FB222720F90E
:102DB00091E0922790FB82F990FB83F92CC08091DF
:102DC0003602982F909591708E7F892B90FB81F918
:102DD0008093360222C00E94380A8091350287FB18
:102DE000222720F991E0922790FB87F914C081E017
:102DF0000E944F1112C08091350284FB222720F9D6
:102E000091E0922790FB84F906C080913502982FBB
:102E1000909590FB80F980933502809135029091D6
:102E200036020E94C9100E94380A80E001C081E089
:102E3000DF91CF910895CF93C82F1F928F938EE883
:102E400091E09F938F930E949F0481E090E0A0E027
:102E5000B0E0BC01CD0104C0660F771F881F991F29
:102E6000CA95D2F70E94900A0F900F900F900F9082
:102E7000CF910C94380AEF92FF920F931F93CF9348
:102E8000DF938B3109F4EDC008F08EC08B3009F46C
:102E9000B1C008F078C0863009F4AFC020F48530A6
:102EA00009F4BDC04EC1873009F4C0C0883009F0B4
:102EB00048C10E94B4101F928F938CE995E09F93B4
:102EC0008F930E949F040E94B01083FB992790F972
:102ED0001F929F9382FB992790F91F929F9381FBEA
:102EE000992790F91F929F93982F91701F929F930B
:102EF0001F928F9383E595E09F938F930E949F0489
:102F00000E94B81087FB222720F91F922F9386FB7F
:102F1000222720F91F922F9385FB222720F91F9249
:102F20002F9384FB222720F91F922F9383FB2227C4
:102F300020F91F922F9382FB222720F91F922F93B3
:102F400091FB222720F91F922F93292F21701F9286
:102F50002F9381FB222720F91F922F93282F217076
:102F60001F922F939F938F938EE694E09F938F935E
:102F70000E949F048DB79EB788960FB6F8949EBFA7
:102F80000FBE8DBF35C0803109F495C020F48E305E
:102F900009F47BC0D6C0863109F4A8C0893109F094
:102FA000D0C08EEF91E084C08A32E1F060F48732C5
:102FB00009F4C3C028F48E3108F4C3C08D51BEC0DB
:102FC000893269F1BEC0833448F48A3308F0B3C053
:102FD000853309F4B2C0883369F0B3C0833409F48F
:102FE000ACC0AFC087E496E00E9406040E944D1179
:102FF000C1E0ACC08BEC92E05BC080911202817F9B
:103000008E7F8093120280EB92E00E94060483E49C
:1030100096E00E94060481E080931602E9CF87E2E1
:1030200096E00E9406040E943F05E2CF80911202C2
:10303000C82FC095C170C0FB80F980931202CC23C9
:1030400029F08BE196E00E94060480C08EE096E0B5
:103050000E94060480911202897F877F809312026A
:10306000C7CF9091120291FBCC27C0F981E0C8270D
:10307000892FC0FB81F980931202CC2319F081E0E3
:1030800096E029C083EF95E013C09091120292FB65
:10309000CC27C0F981E0C827892FC0FB82F9809333
:1030A0001202CC2319F084EE95E015C084ED95E072
:1030B0000E9406049DCF9091120293FBCC27C0F989
:1030C00081E0C827892FC0FB83F980931202CC23AB
:1030D00051F088EC95E00E94060480911202816014
:1030E0008093120233C08BEB95E0E2CF0E94CE1C9E
:1030F000162F072FF82EE92ED0913402C0912B0104
:103100000E94591BEF92FF920F931F931F92DF9320
:103110001F92CF931F928F9383E991E09F938F9398
:103120000E949F048DB79EB70C960FB6F8949EBF71
:103130000FBE8DBF5DCF895301C080E00E941B1779
:1031400057CF89EB95E00E940604C0E08C2FDF91F9
:10315000CF911F910F91FF90EF90089580E0089517
:103160000C94AE18CF93C82F80911602882319F0C3
:10317000813031F038C00E94AB0F8232B1F504C00B
:103180000E94AB0F823261F48C2F0E94B018811123
:1031900004C08C2F0E943B1724C081E090E021C026
:1031A0008C2F0E94AE1881111BC0C43189F018F415
:1031B000CB3029F010C0C93259F0C83361F480EB2C
:1031C00092E00E9406048AE891E00E94060408C08A
:1031D000109216020CC088E891E00E94060407C015
:1031E00081E0817006C01092160280E002C080E08B
:1031F000F8CFCF910895CF93DF9386319C4541F569
:10320000EB010E94AB0F982F8A8120911B01309116
:103210001C01882379F09A7A81E009F480E0809398
:103220001702911102C069E201C065E3C9010E9461
:103230001C1C0AC080911702811102C069E201C002
:1032400065E3C9010E941E1C0E94F00F80E001C0CE
:1032500081E0DF91CF9108950F931F93CF93DF9378
:10326000C42FD22FFC0182818823C9F040931A0217
:103270000E94C21C909319028093180280E28C0F66
:10328000883008F057C0C77081E001C0880FCA9528
:10329000EAF7DF91CF911F910F910C94A4078091D1
:1032A0001A02481330C080911802909119020E94AE
:1032B000DA1C883C910538F510E21D0FCD17B9F0E6
:1032C00080E28C0F883040F4C77081E001C0880F25
:1032D000CA95EAF70E94AB07183028F581E09D2FC8
:1032E000977001C0880F9A95EAF70E94A407802F73
:1032F0000E949B071830F0F4D77081E001C0880F5E
:10330000DA95EAF70AC080E28C0F883098F4C7702B
:1033100081E001C0880FCA95EAF7DF91CF911F9134
:103320000F910C94AB07802FDF91CF911F910F91DC
:103330000C949B07DF91CF911F910F9108950F93EC
:103340009C01CB01243F4CE5340731F188F4293D41
:10335000FCE53F07D9F02A3D4CE5340779F1283DDB
:103360003C45A9F506E221EE41EE68ED7CE52BC077
:10337000263FFCE53F07E1F0A8F0273F3C4539F543
:1033800007E225EE46EE67EF7CE51DC007E225EE7D
:1033900045EE69ED7CE517C006E221EE40EE64EFF4
:1033A0007CE511C007E225EE44EE65EF7CE50BC03D
:1033B00006E221EE42EE66EF7CE505C008E221E080
:1033C00045EE6AED7CE50E942C1980E008C0FC0106
:1033D0008281882319F010921A0201C081E00F91B6
:1033E0000895CF93DF93EC0181E0898B8F810E9458
:1033F000AE0F88850E94C10F0E94F00FEA81FB8109
:10340000CE010696309729F06C897D89DF91CF91A6
:103410000994DF91CF910895EF92FF920F931F933C
:10342000CF93DF93FC012285211136C0EC01E380AC
:10343000F480F7E5FF1A26E12E9DC0012F9D900D27
:103440001124DC01A050BF4F1496ED91FC9115970B
:103450008A5F9E4F309729F054966D917C915597D5
:10346000099586E18E9D80018F9D100D11240050DD
:103470001F4FF80187810E94B40FF80180850E94D8
:10348000C70F0E94F00F188219861B861E821D82AC
:1034900010921C0210921B02DF91CF911F910F918D
:1034A000FF90EF900895DF92EF92FF920F931F939A
:1034B000CF93DF93FB0122812223C1F120911D01D3
:1034C00030911E012F3F3F4F89F18C01C0E0D1E0C8
:1034D000E12CF12CDD24D39480911D0190911E01EB
:1034E0008E159F051CF18E818823D9F089859A85D8
:1034F0008017910739F480911B0290911C020817E4
:10350000190779F0DF861C870B878989811103C031
:10351000CE010E94F119CE0106960E940C1A0E945B
:10352000CE0F4FEFE41AF40A6696D6CFDF91CF9113
:103530001F910F91FF90EF90DF900895EF92FF920F
:103540000F931F93CF93DF939C0137552F3F310586
:1035500011F008F048C040911D0150911E01421722
:10356000530724F430931E0120931D01FB017C01BD
:10357000828196E1929F8001939F100D1124E801B2
:10358000C050DF4F888B92818E81992311F1FA868A
:10359000E9868F5F8E830E94C21C9E878D870E9462
:1035A000D10F8F830E94AB0F88870E94BE0F988532
:1035B000892B8887E881F981C8018A5F9E4F3097FF
:1035C00019F06C897D890995F0921C02E0921B022A
:1035D0000AC0882341F08989882329F0C8018A5FBD
:1035E0009E4F0E940C1A81E0DF91CF911F910F91A5
:1035F000FF90EF900895CF92DF92EF92FF920F939A
:103600001F93CF93DF9380911D0190911E0101962E
:10361000E9F1F12C96E1E92E0F2D10E080911D01CA
:1036200090911E01801791078CF1E09EF001E19EC0
:10363000F00D1124E050FF4FC288D388C114D1048B
:1036400019F488ECC82ED12CE09EE001E19ED00D4B
:103650001124C050DF4F8E818823B1F08D859E8567
:103660000E94DA1CC816D90678F48989811103C032
:10367000CE010E94F119E09EC001E19E900D11243F
:103680008A5F9E4F0E940C1AF394C6CFDF91CF91B0
:103690001F910F91FF90EF90DF90CF90089590933E
:1036A000A5018093A40108959093220280932102A2
:1036B0000895E0912102F0912202309721F00190CB
:1036C000F081E02D099480E00895EF92FF920F932E
:1036D0001F93CF93DF93E0912102F0912202309764
:1036E000B1F18C010280F381E02D099580911202E5
:1036F00082FF2DC080FF04C080E696E00E94060491
:10370000E80118E08AE5E82E86E0F82E80911202A2
:1037100080FF0BC088811F928F93FF92EF920E94CF
:103720009F040F900F900F900F9011502196111140
:10373000EDCF8091120280FF0AC088E596E0DF910C
:10374000CF911F910F91FF90EF900C940604DF91A1
:10375000CF911F910F91FF90EF90089520911F023C
:10376000309120022817390771F09093200280933E
:103770001F02E0912102F0912202309721F0068091
:10378000F781E02D0994089520911D0230911E02C9
:103790002817390771F090931E0280931D02E09163
:1037A0002102F0912202309721F00084F185E02D72
:1037B00009940895FC01329697E080E0915029F039
:1037C00021912223D9F38F5FF9CF0895662349F021
:1037D000FC01329608962191621729F0E817F90743
:1037E000D1F780E0089581E008959C01FC013296B4
:1037F0009FEF80E04191461789F09F3F19F44111F6
:1038000001C0982F8F5F8630A9F79F3F39F0F901EB
:10381000E90FF11D97FDFA956283089508959C01C3
:103820002A5F3F4FFC014281461301C0128201967C
:1038300082179307B9F708950C94F51B0C940F1C8D
:10384000029626E0FC0111922A95E9F70895089561
:103850000C94271C83E0809323020C94281C811174
:1038600002C081E001C082E0809323020C94281CF6
:103870000C942F1C81E0809323020C94281C0C9440
:103880003A1C08950C94411C0C94421C0C94411C4D
:103890000C94411C0C94411CCF930E94481C0E9424
:1038A00041150E94461CC0E08C2F0E943E148111DD
:1038B00004C0CF5FC430C1F701C081E0CF9108954B
:1038C00008951F920F920FB60F9211248F939F931A
:1038D000AF93BF9380912402811113C080913F0266
:1038E00090914002A0914102B09142024196A11DE7
:1038F000B11D80933F0290934002A0934102B09388
:103900004202BF91AF919F918F910F900FBE0F9088
:103910001F90189580914702843031F10E94CA05AA
:103920001092240220E488E190E00FB6F894A89564
:10393000809360000FBE2093600083B7817F846016
:1039400083BF83B7816083BF7894889583B78E7F68
:1039500083BF0FB6F894A89580916000886180932A
:103960006000109260000FBE08950E94380A0C9407
:10397000CE0582E084BD93E095BD9AEF97BD80931C
:103980006E0008952FB7F89480913F029091400205
:10399000A0914102B09142022FBF08952FB7F89431
:1039A00060913F02709140028091410290914202E9
:1039B0002FBF08959C014FB7F89480913F029091DA
:1039C0004002A0914102B09142024FBF821B930B73
:1039D000089578941F920F920FB60F9211248F932F
:1039E0009F93AF93BF9380913F0290914002A0912B
:1039F0004102B09142020196A11DB11D80933F0288
:103A000090934002A0934102B0934202BF91AF91C4
:103A10009F918F910F900FBE0F901F90189587E781
:103A200097E790930108809300089AE088E10FB629
:103A3000F894A895809360000FBE90936000FFCF2C
:103A40008091330208950895CF93DF9321E020936E
:103A5000E9002FEF3091E800215035FD06C035ED2B
:103A60003A95F1F700002111F5CF2091E80025FFEC
:103A700014C0EC0140E050E068E070E00E94EE1FEE
:103A80008091E8008E778093E80088E0FE01ABE249
:103A9000B2E001900D928A95E1F7DF91CF91089500
:103AA0008093270270932902609328028091470235
:103AB000843001F582E08093E9008FEF9091E80077
:103AC000815095FD06C095ED9A95F1F700008111A2
:103AD000F5CF8091E80085FF0DC040E050E063E045
:103AE00070E087E292E00E94EE1F8091E8008E77FE
:103AF0008093E8000895BC0184E00C94501DBC0143
:103B000083E00C94501D089586E896E00E94060418
:103B100080914602811109C00E947F210E94DC2110
:103B20008091E20084608093E200089582E896E04C
:103B30000E9406041092460208958EE796E00E94C5
:103B400006040C943F1C8AE796E00E9406046091EC
:103B5000430281E0611101C080E00C942A1C86E7D9
:103B600096E00E9406049091470281E0943009F0AB
:103B700080E0609143020C942F1C209126022F5F5D
:103B8000822F62E30E948B24992319F0209326024E
:103B900008951092260280912A02882371F1809163
:103BA0004702843041F58091E9008F702091EC004C
:103BB000922F917020FD90E8892B93E09093E9007B
:103BC0009091EB0090FF14C09091EE0097FF10C011
:103BD0009091E80095FF03C01092F100F9CF909109
:103BE000E80090FF05C09091E8009E779093E80070
:103BF0008F708093E90010922A02089542E061ECF0
:103C000081E00E94F82042E261EC82E00E94F8200C
:103C100042E261EC83E00E94F8209091470281E04B
:103C2000943009F080E0609143020C94381C80913C
:103C30004902833009F461C030F4813071F0823080
:103C400009F49AC008958A3009F486C08B3009F4CB
:103C50006CC0893009F0A8C020C080914802813A28
:103C600009F0A2C08091E800877F8093E8008091EE
:103C70004C0290914D02892B21F468E08BE292E096
:103C800003C060E080E090E070E00E943920809105
:103C9000E8008B778093E800089580914802813294
:103CA00009F082C080914C0290914D02029708F079
:103CB0007BC08091E800877F8093E8008091E800D6
:103CC00082FD05C0809147028111F8CF6DC020911F
:103CD000F3008091F20090E0922B029731F48091F2
:103CE000F100813011F0863021F48091F100809351
:103CF00033028091E8008B7753C080914802813A6B
:103D000009F052C080914C0290914D02892B09F02C
:103D10004BC08091E800877F8093E8008091E800A5
:103D200080FFFCCF80912B0136C080914802813208
:103D3000D9F580914C0290914D02892BA9F5809183
:103D4000E800877F8093E8000E942D2180914A023D
:103D500080932B010C94380A80914802813221F51E
:103D60008091E800877F8093E8000E942D21809158
:103D70004B0280933402089580914802813AA1F465
:103D80008091E800877F8093E8008091E80080FFC1
:103D9000FCCF809134028093F1008091E8008E770F
:103DA0008093E8000C942D2108959FB7F894109209
:103DB0002A029FBF90914702943009F057C090911A
:103DC000E9009F703091EC00232F217030FD20E836
:103DD000922B23E02093E9002091EB0020FF43C0C9
:103DE0002091EE0027FF3FC020912502222321F0E1
:103DF0002091E80025FF37C01092250226E030917F
:103E0000E80035FD15C030914702343061F530913E
:103E1000EB0035FD28C0215021F481E0809325027C
:103E200022C0EFE9FFE03197F1F700C00000E7CFD3
:103E30008093F1008091E80085FD0AC08091E80040
:103E400080FFFCCF8091E8008E778093E80006C069
:103E50008FB7F89421E020932A028FBF9F70909330
:103E6000E90080E008959F709093E9008FEF089536
:103E700084B7877F84BF0FB6F894A89580916000BF
:103E8000886180936000109260000FBE90E080E82F
:103E90000FB6F89480936100909361000FBE0C946C
:103EA0003A1C0E947F210E94DC21E2EEF0E080813A
:103EB0008460808378940C9470248FE191E00C945A
:103EC000541B809147028530C9F482E796E00E9436
:103ED000060480914702853079F40E948A1C809103
:103EE00045028823B1F30E944C1C882391F30E9461
:103EF000D81F0E94380AEDCF0C94B51C0895089580
:103F00000C94821F292F332723303105C9F060F428
:103F10002130310581F02230310509F041C08BE5B7
:103F200090E024EB36E040C021323105E1F022324E
:103F3000310531F135C082E190E02FE037E034C047
:103F400099278130910549F028F0029749F5EAE870
:103F5000F6E005C0E0EBF6E002C0EAE9F6E08491A5
:103F600090E09F0121C063307105D0F4660F771F88
:103F7000FB01E256FE4F2081318189E090E014C0C0
:103F80006330710568F4FB01EE0FFF1FE856FE4F2A
:103F900020813181FB01EB56FE4F808190E004C00F
:103FA00080E090E020E030E0FA0131832083089542
:103FB00080E189BD82E189BD09B400FEFDCF809119
:103FC000D8008F7D8093D8008091E000826080933C
:103FD000E0008091E00081FDFCCF0895CF92DF9258
:103FE000EF92FF920F931F93CF93DF93EC018B011E
:103FF0007A010E944C21811133C0E114F10439F09F
:10400000F70180819181081B190BC80FD91FC12CA2
:10401000D12C0115110519F18091E80085FD16C01C
:104020008091E8008E778093E800E114F10449F074
:10403000F70180819181C80ED91ED182C08285E0AE
:104040000FC00E944C21882321F30AC089918093DC
:10405000F10001501109FFEFCF1ADF0ADACF80E03B
:10406000DF91CF911F910F91FF90EF90DF90CF9054
:10407000089520914E0230914F022617370748F0DD
:104080006115710539F42091E8002E772093E8003E
:1040900001C0B901FC0120E06115710579F1809141
:1040A00047028823F1F18530F1F18091E80083FD2A
:1040B0003CC08091E80082FD2EC08091E80080FF26
:1040C000EBCF2091F3008091F20090E0922B6115EC
:1040D000710551F08830910538F421912093F10059
:1040E000615071090196F3CF21E0089709F020E0B3
:1040F0008091E8008E778093E800CECF2111CFCF5A
:104100000AC080914702882361F0853061F0809178
:10411000E80083FD0AC08091E80082FFF2CF80E0D2
:10412000089582E0089583E0089581E00895209144
:104130004E0230914F022617370748F0611571057E
:1041400039F42091E8002E772093E80001C0B901EE
:10415000FC0120E06115710591F1809147028823EF
:1041600009F440C0853009F43FC08091E80083FD28
:104170003DC08091E80082FD2FC08091E80080FF63
:10418000E9CF2091F3008091F20090E0922B61152D
:10419000710559F08830910540F424912093F10085
:1041A0003196615071090196F2CF21E0089709F02C
:1041B00020E08091E8008E778093E800CBCF21113A
:1041C000CCCF0AC080914702882361F0853061F02E
:1041D0008091E80083FD0AC08091E80082FFF2CF61
:1041E00080E0089582E0089583E0089581E00895D5
:1041F000982F973068F59093E900981739F07091EF
:10420000EC002091ED005091F00003C0242F762F98
:1042100050E021FD02C09F5FECCF3091EB003E7F6C
:104220003093EB003091ED003D7F3093ED00309105
:10423000EB0031603093EB007093EC002093ED00C5
:104240005093F0002091EE0027FDE5CF80E0089527
:104250008F708093E90081E008958091480287FF84
:1042600011C08091E80082FD05C080914702811154
:10427000F8CF11C08091E8008B770BC08091470286
:10428000882349F08091E80080FFF8CF8091E80012
:104290008E778093E80008952091E4003091E50046
:1042A00095E64091EC00842F817040FF23C08091FF
:1042B000E80080FD1DC080914702882399F0853079
:1042C00099F08091EB0085FD11C04091E400509180
:1042D000E5002417350729F3915011F09A01E1CF39
:1042E00084E0089582E0089583E0089581E00895D0
:1042F00080E008954091E80042FFDDCF08950E94DC
:10430000ED210E94F521E0EEF0E080818160808364
:10431000E8EDF0E080818F77808319BCA7EDB0E0F5
:104320008C918E7F8C9380818F7E80831092460249
:1043300008950F931F93CF93DF930E94ED210E9466
:10434000F521C8EDD0E088818F77888388818068E7
:10435000888388818F7D888319BC109247021092D0
:104360004302109245021092440200EE10E0F80160
:1043700080818B7F808388818160888342E060E0D8
:1043800080E00E94F820E1EEF0E080818E7F808363
:10439000E2EEF0E0808181608083808188608083AC
:1043A000F80180818E7F8083888180618883DF919E
:1043B000CF911F910F910895E8EDF0E080818F7EFD
:1043C0008083E7EDF0E080818160808384E082BFBC
:1043D00081E0809346020C949921E8EDF0E0808121
:1043E0008E7F80831092E20008951092DA0010927E
:1043F000E10008951F920F920FB60F9211242F9390
:104400003F934F935F936F937F938F939F93AF935C
:10441000BF93EF93FF938091E10082FF0BC08091E7
:10442000E20082FF07C08091E1008B7F8093E10072
:104430000E94BD1D8091DA0080FF1FC08091D800CE
:1044400080FF1BC08091DA008E7F8093DA0080911C
:10445000D90080FF0DC080E189BD82E189BD09B42A
:1044600000FEFDCF81E0809347020E94841D05C0BD
:1044700019BC109247020E94961D8091E10080FFB6
:1044800019C08091E20080FF15C08091E2008E7F0C
:104490008093E2008091E20080618093E20080914D
:1044A000D80080628093D80019BC85E080934702D1
:1044B0000E94A31D8091E10084FF30C08091E20042
:1044C00084FF2CC080E189BD82E189BD09B400FE72
:1044D000FDCF8091D8008F7D8093D8008091E1003E
:1044E0008F7E8093E1008091E2008F7E8093E200D6
:1044F0008091E20081608093E200809143028823F2
:1045000011F084E007C08091E30087FD02C081E0E4
:1045100001C083E0809347020E94AF1D8091E100BB
:1045200083FF29C08091E20083FF25C08091E100D4
:10453000877F8093E10082E08093470210924302DC
:104540008091E1008E7F8093E1008091E2008E7F78
:104550008093E2008091E20080618093E20042E07B
:1045600060E080E00E94F8208091F00088608093F5
:10457000F0000E949D1DFF91EF91BF91AF919F911F
:104580008F917F916F915F914F913F912F910F90FC
:104590000FBE0F901F9018951F920F920FB60F929B
:1045A00011242F933F934F935F936F937F938F9338
:1045B0009F93AF93BF93CF93DF93EF93FF93C091FC
:1045C000E900CF708091EC00D82FD17080FDD0E849
:1045D0001092E9008091F000877F8093F00078943A
:1045E0000E9410231092E9008091F000886080936F
:1045F000F000CD2BCF70C093E900FF91EF91DF91D8
:10460000CF91BF91AF919F918F917F916F915F916A
:104610004F913F912F910F900FBE0F901F901895C3
:104620001F93CF93DF93CDB7DEB7AA970FB6F89459
:10463000DEBF0FBECDBFE8E4F2E08091F1008193D0
:1046400022E0E035F207C9F70E94171E8091E800CA
:1046500083FF2EC18091480290914902492F50E07A
:104660004A30510508F024C1FA01EE59FF4F0C946D
:104670009724803821F0823809F01AC108C080914F
:10468000440290914502992389F082600FC0809185
:104690004C028F70873008F00BC18093E900809145
:1046A000EB0085FB882780F91092E9009091E800E3
:1046B000977F9093E8008093F1001092F100D1C0B1
:1046C000282F2D7F09F0F4C0882319F0823061F083
:1046D000EFC080914A02813009F0EAC0933009F0BE
:1046E00080E0809345022EC080914A0281112AC049
:1046F00080914C028F702FEF280F263008F0D8C021
:104700008093E9002091EB0020FF1CC0933021F43E
:104710008091EB00806214C09091EB0090619093C7
:10472000EB0021E030E0A90102C0440F551F8A953B
:10473000E2F74093EA001092EA008091EB00886073
:104740008093EB001092E9008091E800877F8093CE
:10475000E8000E942D21ACC08111AAC010914A022C
:104760001F778091E3008078812B8093E300809114
:10477000E800877F8093E8000E942D218091E80067
:1047800080FFFCCF8091E30080688093E3001111EB
:1047900002C082E001C083E08093470289C0805854
:1047A000823008F085C080914A0290914B028C3D86
:1047B00053E0950779F583E08A838AE289834FB7CE
:1047C000F894DE01139620E03EE051E2E32FF0E0A2
:1047D00050935700E49120FF03C0E295EF703F5FD4
:1047E000EF708E2F90E0EA3010F0C79601C0C096AF
:1047F0008D939D932F5F243149F74FBF8091E8003F
:10480000877F8093E8006AE270E0CE0101960E9403
:10481000392016C060914C0270914D02AE014F5F7D
:104820005F4F0E94801FBC01892B09F441C0909109
:10483000E800977F9093E80089819A810E949720F1
:104840008091E8008B778093E80032C0803881F552
:104850008091E800877F8093E800809143028093F5
:10486000F1008091E8008E7772CF811121C0809194
:104870004A0290914B0299270297D4F48091E80064
:10488000877F8093E80080914A02809343020E94D0
:104890002D2180914302811106C08091E30087FDA4
:1048A00002C081E001C084E0809347020E94FE1DA7
:1048B0008091E80083FF0AC08091E800877F8093A1
:1048C000E8008091EB0080628093EB00AA960FB61F
:1048D000F894DEBF0FBECDBFDF91CF911F91089539
:1048E000CF93809147028823A1F0C091E900CF7057
:1048F0009091EC00892F817090FD80E8C82B109278
:10490000E9008091E80083FD0E941023CF70C093DE
:10491000E900CF910895991B79E004C0991F96177B
:1049200008F0961B881F7A95C9F780950895EE0FB9
:10493000FF1F0590F491E02D0994FB01DC0104C0F8
:104940008D910190801921F441505040C8F7881B87
:10495000990B0895F999FECF92BD81BDF89A9927D8
:1049600080B50895A8E1B0E042E050E00C94DE2468
:10497000262FF999FECF92BD81BDF89A019700B418
:10498000021639F01FBA20BD0FB6F894FA9AF99AB8
:104990000FBE08950396272F0E94B9240E94B824C1
:1049A000252F0E94B924242F0C94B9240196272F77
:1049B0000E94B9240C94B824DC01CB01FC01F999C4
:1049C000FECF06C0F2BDE1BDF89A319600B40D925B
:0C49D00041505040B8F70895F894FFCF14
:1049DC000000CA04AC04000000000000000000004D
:1049EC00000013010000010000C800FC01FFFF20C3
:1049FC001D241D831D7F1D7B1D231D01E200E9006D
:104A0C00EA00B500B600B700CD008301CC008A01E6
:104A1C00920194012102230224022502260227027C
:104A2C002A02B300B4006F007000818283E200E9B7
:104A3C0000EA00B500B600B700CD008301CC008AB7
:104A4C00019201940121022302240225022602274D
:104A5C00022A02B300B4006F007000818283946656
:104A6C003136323334403222750743072107C606EC
:044A7C00DF06F80653
:00000001FF
